:020000000130CD
:02000B0021E1F1
:10003000758902D2A9D2AF758C06758A0075816F59
:10004000D2B9D28C7590FF75B0FF75300075310054
:10005000754200C209C20BE52664227025E54164A1
:1000600038701FB210300B2EE5324533453445351C
:1000700054F07010853236853337853438853539FC
:1000800001A2C21075360075370075380175390048
:100090007526227541388536328537338538348563
:1000A0003935C20BC208C20AD2B7753D78753EC851
:1000B000753F01514C3009FD317F11F2300A0211B8
:1000C000E5200BA130B20201B530080280E775309F
:1000D00000753100754200D208C20AC210C20B512D
:1000E0004CC2B780D0C2AF7590FF75B0FF43870296
:1000F000002230080122D53D0E753D78D53E0875A9
:100100003EC8D53F0280DEA2B3500A753C0E753A58
:1001100001753B0A22D2B7C208C20AD53CF6753C2B
:100120000ED53AF0853B3A153BE53BB40102053B61
:10013000D20B201024E53564097007E5346409709A
:100140000122E525B43202415E753200B43302412A
:1001500068753200B434EA4168E5326401700945DB
:100160003345344535700122E525B4320241277507
:100170003200B433024131753200B434EA41310502
:1001800020C209519B74035520F5202432F8E63033
:100190000E0224109001C193300F0274FF43B0335C
:1001A000F590E5207003C2B422147006201611C227
:1001B000B522147006201508C2B122201402C2B064
:1001C0002214B78C85274544970405FFFFFFFFFFE6
:1001D000EF10B38881234140930001FBFBFBFBFB45
:1001E000FFC0E0C0D00530740AB530366230D209A5
:1001F000053174C8B5312B6231B20C200B24300CA0
:10020000210542743CB5421A6242300815E53214A9
:100210004534453345357008C208D20AD2B7412269
:100220005127D0D0D0E0321532E532F4701E75324D
:10023000091533E533F470147533051534E534F4DA
:10024000700A7534091535E535F47000752534E507
:1002500035700A752533E534700375253222053271
:10026000740AB5322475320005337406B5331A7535
:1002700033000534740AB534107534000535740A3A
:10028000B53506753509753409752534E535700AB7
:10029000752533E534700375253222C216C215C2A6
:1002A00014E535700ED214E5347008C215E53370CC
:1002B00002C216E520C20EB40202D20E300808A215
:1002C0000C820E920E800AA20C920FC20F30B30164
:0402D00022C20F2215
